S123E0007EED77BDECFAFEFFC4A60A815526040EBDF15EBDE068FCFFC0F3FFC28F350E4F57
S123E0205FDD3ADD3FDD41BDE0AB7F00197F00187F001DBDE105BDE0BBBDE05BBDEE4D1A14
S123E04083000026D1DE0ADF2FBDE1277D001926C520D7DE2F6F00DF0A20BBBDE3C38120CB
S123E0602605BDE3CC20F439CEE06E7EE11C0D0A0D0A424153494331312076312E35350DC3
S123E0800A436F7079726967687420313938352D313939302062790D0A476F72646F6E2027
S123E0A0446F7567686D616E0D0A00CEE0B17EE11C0D0A52454144590D0A00C64FDE49BD9C
S123E0C0FEEF810D272B5D272881082610C14F2720098620BDFED28608BDFED25C81032650
S123E0E0067C001C7EF274812025D4A700085A26CE860DA700DE49DF003981612506817A82
S123E100220284DF39CEE10A20120D0A23008D00CEE1198D077F001E390A0D00A60027066D
S123E120BDFED20820F639DE4BDF028D3F241936BDE3C3810D322609BDEBA1DE0A08DF2D17
S123E140397F00198D6E2010BDE3C3810D27F186019719CC000020ECBDE1E27D0019270367
S123E1607EF233BDEB7ADE0A08DF2D39183C4F36361830DE00A6008D422410A6008D3C252F
S123E180110D18EC0026048612200D31311838DF00398D072AE586017EEA9818EC00050568
S123E1A018E3000518ED00E60008C0304F18E30018ED0039BDE3D44F7EE3D7813025068198
S123E1C03922020D390C398141250E815A230881612506817A22020D390C398DEA240139CC
S123E1E020D9BDE3C3810D274F7F001ABDE37ACEE246BDE3A5251308A60026FBC6043A6D55
S123E2000026EF8602CEE41C2004A601EE02BDE3D7810C2707810A2703BDE37AAD00BDE386
S123E2207ABDE3CA813A2607867ABDE3D720B3810D270586027EEA98867DBDE3D7DC029397
S123E2404BDE4BE7023944415441000CE3FC4C45540001E41C52454144000DEA58524553E4
S123E260544F5245000EE3FB474F535542000FE3F2474F544F0012E3F24F4E54494D450024
S123E28025E8D34F4E4952510026E8D34F4E504143430028E8F34F4E0013E885524554551C
S123E2A0524E0014E3FB49460015E907494E5055540016EA405052494E540003E9D83F00D4
S123E2C003E9D8464F520004E9704E4558540005E9CB53544F500017E3FB454E4457480089
S123E2E01AE3FB454E440018E3FB52454D000AE3FC54524F4E0006E3FB54524F46460007D9
S123E300E3FB5748494C450019EA8B504F4B450008E7FA44494D0009EA58454550001BE8FA
S123E32013504F525441001CE418504F525442001DE418504F525443001EE418504F5254A1
S123E34044001FE418494E425954450023EA8354494D450024EA93524554490027E3FB50A6
S123E360414343000BEA93534C4545500029E3FB5254494D45002AE3FB003CDE005FA60022
S123E380812026045C0820F65D26023839DF00DE02C101270C867FA70008E70008DF0238CE
S123E3A039C67E20F5DC003736A60027128D1BBDE0FAA10027063233DD000C390820EA32C7
S123E3C0330D393CDE00A60038398DF73CDE0008DF0038398D01173C3736DE02A70008DFDD
S123E3E002DC4BC300801A9302323322E586147EEA9886A88DE1BDE16C20D939DE023C867E
S123E400008DD4C6028DBC810D27078DCA8DBD5C20F38DC338E70039C6012004BDE5571618
S123E4208DA8813D270586037EEA9886798DA817183C361830CEE54EBDE4FD24028D98BD6C
S123E440E3C381282622BDE3CC8610BDE3D718A600BDE430BDE3CA8129270586047EEA984F
S123E4608611BDE3D77EE497BDE1BB25088124270481222605BDE66C2009BDE7674D2603B4
S123E480BDE55718E600C100260318A70018A100270586057EEA98BDE3C3810D2740813A55
S123E4A0273C81202738812C2734813B27308129272C18A60081012618BDE4E82518BDE4F8
S123E4C0F325137D001A2705BDE4F820098600200586137EEA984D260986067EEA983118F3
S123E4E03839BDE3D77EE435CEE513BDE4FD2502860039CEE52320F3CEE53820EEBDE3A528
S123E500250D08A60026FB0808A60026F00C39A6010D392B00402D00412A00502F00515CC9
S123E5200052002E414E442E00202E4F522E00212E454F522E0022003C3D00323E3D00335B
S123E5403C3E00353C00303E00313D0034002D00724E4F54007100183C4F363636361830F8
S123E560BDE3C3BDE1C7250586077EEA98BDE0FA18A700BDE3CCBDE3C3BDE1DB2409BDE0B0
S123E580FA18A701BDE3CCBDE5E018A703BDE5EE1A83FFFF260618A603BDE626373618A601
S123E5A003BDE3D73233BDE3D418A6038510271EBDE3CC8610BDE3D78601BDE430BDE3CA2E
S123E5C081292705860E7EEA988611BDE3D7860118E603C502270286023131313118383972
S123E5E0868436BDE3C381283226028B1039DE086D00272EA1002612E60118E100260BE625
S123E6000218E10126048F930839E600C5102704C6052006C1842605C6053A20D386087E22
S123E620EA98CCFFFF39DE0A3CA7000818E600E7000818E601E700088D186F00DF0A9C10FA
S123E640230486092023323393083736BDF2E332333985102704C602200681842609C60276
S123E6606F00085A26FA3986087EEA98BDE3C3DE003C81242608BDE3CCBDE6CF2003BDE6EA
S123E680A13686A4BDE3D732BDE3D4DC0030A30017BDE3D738A600BDE3D7085A26F78601C0
S123E6A039183C4F36361830DE00A600BDE1BB25048602202CA600BDE1BB2409BDE19B2A5D
S123E6C0F4860A201CDF0018EC003131183839183C4F36361830DE00A600BDE721250D8650
S123E6E00B7D001D27037EEAEF7EEA98A600BDE72124D218EC0005252405252105251E05A5
S123E700251B18ED00A600BDE0FA1608C030C1092302C0074F18E30018ED0020CF860C20BF
S123E720C0BDE1BB240139BDE0FA81412506814622020D390C39C60286A2BDE3D7DE023CE1
S123E7404FBDE3D7BDE3CABDE3D7BDE3CA8122270F810D2605860D7EEA98BDE3D75C20EAA2
S123E760BDE3D738E70039CEE788BDE3A5250E08A60026FBC6043A6D0026EF4F398636BDBB
S123E780E3D7A601EE026E00464449560001E801434852240002E81F4142530004E81F5266
S123E7A04E440005E81F53474E0006E81F5441420007E81F4144430003E81F43414C4C00EF
S123E7C008E81F5045454B0009E81F454550000AE81F484558320012E81F484558000BE8FE
S123E7E01F504F5254000CE86854494D450011E87F504143430013E87F00DE0209DF02A6AD
S123E80000183CC60137371830C602BDE82E3232183839DE0209DF02A6008D037EE4201801
S123E8203CC60137C60118308D0432183839BDE3D7BDE3C381282705860E7EEA98BDE3CC90
S123E8408610BDE3D718A600180837BDE430335A2707BDEA2D24E120ECBDE3C3812926D816
S123E860BDE3CC86117EE3D7BDE3CABDE0FA81412405862F7EEA98814522F780418B0CBDC4
S123E880E3D78601398601BDE430BDE37ACEE271BDE3A5240D8612BDE3D7BDE37ABDE3F236
S123E8A02018CEE268BDE3A52505860F7EEA98860FBDE3D7BDE37ABDE3F2BDE37ABDEA2D5A
S123E8C0250139BDE37A86A8BDE3D7BDE16CBDE3D420E78601BDE430BDE37ABDEA2D250521
S123E8E086157EEA98BDE37A86A8BDE3D7BDE16C7EE3D48D0220DC8601BDE430BDE37ABDC1
S123E900EA2D24DC7EE37A7C001A8601BDE430BDE37ACEE966BDE3A5250586107EEA988651
S123E92038BDE3D7BDE37ABDE3C3BDE1BB242786A8BDE3D7BDE16CBDE3D4BDE37ACEE96BA4
S123E940BDE3A52501398639BDE3D7BDE37ABDE3C3BDE1BB250586127EEA9886A8BDE3D79C
S123E960BDE16C7EE3D45448454E00454C534500BDE5578101270586037EEA98BDE3CA81E1
S123E9803D26F48679BDE3D78601BDE430BDE37ACEE9C3BDE3A5250586117EEA988637BD3A
S123E9A0E3D7BDE37A8601BDE430BDE37ACEE9C6BDE3A5250139863ABDE3D7BDE37A860114
S123E9C07EE430544F005354455000BDE5578101270586027EEA9839BDE3C38123260D869A
S123E9E078BDE3D7BDE3CCBDE37A201BBDE37ABDE3C3810D2704813A260139BDE3C381220C
S123EA002605BDE73620058601BDE430BDE37ABDE3C3810D27E4813A27E08D1125CE813B4B
S123EA20270586167EEA98867B8D0D20BFBDE3C3812C27020C39867CBDE3D7BDE3CC0D39E7
S123EA408D21BDE37ABDE3C38122260CBDE7368DDC250586157EEA98BDE557BDE37A8DCD3D
S123EA6025F639BDE3C381232701398678BDE3D7BDE3CCBDE37A8601BDE430BDE37A8DAD2F
S123EA8024D1398DDEBDE37A7EE5577C001A86007EE430C6017EE4209718BDE10EDE49A6E6
S123EAA000810D2706BDFED20820F4BDE110DE0009099C49230EDF00DE49862ABDFED208EF
S123EAC09C0026F8CEEAE2BDE11CBDE1108D078601971C7EE053CEEAE6BDE11CD6184F7EE4
S123EAE0EB1A5E5E5E004552524F52202320009718BDEAD6CEEB0EBDE11CDC29BDEB1ABDD5
S123EB00E1108601971C7EE016425245414B20494E204C494E45202320001A8300002605C3
S123EB2086307EFED2183C3736CC271037365F37183018EC032A0D4353C3000118ED038698
S123EB402DBDFED218EC03CDEE010218ED038F1A8300002605186D00270B178B30C601186B
S123EB60E700BDFED218EC01CE000A02CDEF0126D3C605183A18351838398601971CDE4B32
S123EB80EC001A930C230ABDEC69DE4BEC00DD0C398D56EC003CDE4B1AA30038266A7EEC33
S123EBA086373618301A930C23078601971C3233398D36EC00CDA30026F0E6028D0DDC0CBC
S123EBC0CDA30026E58D31DD0C20DF183C3C1838183A189C06240A18A600A7000818082049
S123EBE0F1DF06BDECC9183839DE041AA300230737E6023A3320F439DE049C062709EC00FE
S123EC0037E6023A3320F3393CDE4BE602383C8D03382040183C3CDE0A3A9C0E222BBDECDD
S123EC20A3DE063C3A3C183018EC00DD0618EC02CDA3042519CDEE02A60009CDEF02CDEECB
S123EC4000A70009CDEF0020E486097EEA983838381838393CDE4BE6023818DE4B18A600FC
S123EC601808A700085A26F539DE4BE602DE0A3A9C0E220DBDECA3DE063A8FDE06DD062027
S123EC80D386097EEA98E6023CDE4BE00238260220C22A08503CBDEC143820B83CBDEBCB63
S123ECA03820B1183C37DE0A18DE0A3ADC0ADF0A9308270FDD6C18A600A7000918098D3263
S123ECC02AF408DF0833183839183C3718DE0886FF50D3088FDC0A9308DF08DD6C270D18A2
S123ECE0A600A7000818088D092AF409DF0A33183839DC6C830001DD6C39FEFFC0DF08DF68
S123ED000ADF04DF068FF3FFC2830251DD10DD0EC30001DD49C30050DD4BC30080DD4DC3D7
S123ED20001EDD4FDD51C3003CDD53DD55C30050DD57DD59C30010DD5BDD5DC30010DD5F25
S123ED40DE046F00089C0E23F9FEFFC4A60A81552603BDF3AFCC0000DD0CDD29BDF28B7F4D
S123ED60001B8601971CFEFFCEA7007F00377F0019DE0A08DF2D39FCFFC8DD614444444434
S123ED80B7103DDE618693A7398603A724FCFFC0F3FFC28F35CE00C418CEEE00C614867E68
S123EDA0A700081AEF0008085A26F5CE00F7CCED77ED01ED04ED07CE00A418CEFFA0C6206D
S123EDC018A600A7000818085A26F5CEEDFEDFE08603973C4F5FDD38DD3ADE618D2386808A
S123EDE0A722CEEE3BDFEFCEEE41DFCBDFCE4F5FDD3DDD3FDD41FEFFCCAD007EE0038D01C6
S123EE003BDE61EC16F3FFCAED168680A7237A003C26278602973CDC38C30001DD38DC3A82
S123EE2027181A9338261318DE3D31317C0019DC29DD45DC2BDD477EF44A3918DE3F26ECB9
S123EE403BDE618630A72518DE4126E03BBDE3C3810D2604CC000039CEEE76BDE3A5250E70
S123EE6008A60026FB0808086D0026EF20E6EE01AD00CC0001394C49535400EECA52554E94
S123EE8000F15E4E455700F2CC434F4E5400F2B7434C45415200F2E0455341564500F2F704
S123EEA0454C4F414400F35B4C4C49535400F3954155544F535400F3A04E4F4155544F0042
S123EEC0F3AB4652454500F3DC00BDE10EDC041A9306260139BDE05BBDE3C3BDE1BB242701
S123EEE0BDE16CDD12BDE3C3812D270ADC12DD141A930C232139BDE3CCBDE16C1A930C236C
S123EF0002DC0CDD14200F810D270139DE04EC00DD12DC0CDD14DC121A9314230139DC1264
S123EF20BDEBE9DF6ADC14BDEBE9EC001A93142603E6023ADF14DC6A1A9314260139DE6AD8
S123EF40EC00080808DF6ABDEB1ADE6AA600817D270D4D2B05BDEFDD20F0BDEF6920EBBD8B
S123EF60E110DE6A08DF6A20CDDE6AA60084EFCEEF87A100270C0808086D0026F586087EF1
S123EF80EA98EE01AD003984EF94A2EFC9A8EFD0A4EFC200DE6A08EC00D3080808DF6A8FFA
S123EFA0A601BDFED2A6022703BDFED239DC6AC300068FE60008A600BDFED2085A26F7DF64
S123EFC06A39DC6AC3000320E9DC6AC3000120E2DE6A08EC000808DF6ABDEB1A39DE6AA6EB
S123EFE00008DF6A817F26037EF021810A26037EF039810C26037EF0318136260CDE6AA67D
S123F0000008DF6ACEF1102003CEF052A100270C0808086D0026F586087EEA98EE017EE149
S123F0201CDE6AE60008DF6A8620BDFED25A26FA39CEE246BDE11C2006CEE2EABDE11CDE43
S123F0406A08A600810D260408DF6A39BDFED20820F001E24E0DE2550EE25D0FE26812E29E
S123F0607113E29614E29C15E2A638E96639E96B16E2AC03E2B504E2C305E2CA17E2D218D2
S123F080E2E306E2F107E2F919E3021AE2DA3AE9C637E9C37CF14E7BF14C7AF14A02F149E8
S123F0A008E30B79E54A10F15011F15220E52321E52A22E53030E54431E54732E53833E55D
S123F0C03C34E54A35E54040E51341E51650E51951E51C52E51F71E5512AE37072E54E7E82
S123F0E0F15409E3131BE31A1CE3211DE32A1EE3331FE33C78F15C23E34524E34F25E2790E
S123F10026E28327E3570BE35F28E28C29E3670001E78802E79003E7B404E79805E79F060E
S123F120E7A607E7AD08E7BB09E7C30AE31A0BE7DA0CE3210DE32A0EE3330FE33C10F156A0
S123F14011E34F12E7D213E35F003A003B002C00280029002000504F525445002300BDE1EB
S123F1600EBDF28B8601971D18DE04189C0626013918EC00DD297D001B2712865BBDFED2AB
S123F180DC29BDEB1A865DBDFED2BDE110183C18E602183A18DF2B1838C603183A8D30187E
S123F1A0E60018088D295A58CEF1DF3AEE00AD007A001A2603BDF2648D1518A600817D2616
S123F1C00A1808189C0626A97EF4CD180820CE18A6002B0A817E270425041808180839F379
S123F1E0F1F3F1F619F782F7D9F604F609F5BEF711F3EBFA51F3EBF8F9F91CF47E000000AB
S123F20000F43BF55BF4AAF956F819F4BDF4CDF4F1F536F97FF5DEF5F8F5FCF600000000CC
S123F220000000FA22FA34FA66FA7DFA9BFABDF60DFA3FBDE10E18DE4B18EC00DD29C60361
S123F240183A8D8B18E60018088D845A58CEF1DF3AEE00AD00BDF1CF18A600817D26013953
S123F260180820DE860A971A9D9E2601399DA1810327013918DF31BDE110CEEB09BDE11C1B
S123F280DC29BDEB1ABDE1107EE016BDF2E0DE53DF1FDE4FDF21DE57DF23DE5BDF25DE5FE5
S123F2A0DF27DE0A08DF2D7F001E860A971A7F001CCE0000DF3339BDE10E7D001C2606182D
S123F2C0DE317EF1B8862597187EEAD6FEFFC4A60A8155260786FFA70ABDFA19BDECFA3906
S123F2E0BDF28EDE08A6002708080808BDE65220F4DE0A08DF2D39DC041A9306260139DCED
S123F3000A93041AB3FFC6230586377EEA98FEFFC418CE0004C604D71A18EC00B3FFC0A74E
S123F32000BDFA190817A700BDFA1908180818087A001A26E418EC00A700BDFA190817A73C
S123F34000BDFA19FEFFC418DE0418A600A70BBDFA19081808189C0A23F039FEFFC418CE05
S123F3600004C604D71AEC00F3FFC018ED000808180818087A001A26EDEC0018ED00FEFF42
S123F380C418DE04A60B18A700081808189C0A23F318DF2D3986019737BDEECA7F00373929
S123F3A08655FEFFC4A70ABDFA193986FF20F3FEFFC4FCFFC4C3000BDD04FCFFC4E302C3C5
S123F3C0000BDD06EC06A304F3FFC0DD0AFCFFC0DD08188FFCFFC4E3048F20A8BDE10EDC3D
S123F3E010932DBDEB1ABDE110393918E600183A3918A6008D0E37361808BDFB17BDFBBEA3
S123F40038ED003918A6008502261D8510260F18EC01D308C3000337C603183A3339BDFB1C
S123F420953C3005E3003839851027E3BDFB953C37363005E30031313020E97D0019270465
S123F440DC06DD2BDE2B9C062604DE042007EC00CDA30122F5EC00CDA30127102505861B0D
S123F4607EEAEFE6023A9C0627F420E98F188F7D001927067F00197EF1C3313120F9183CB7
S123F4807D0019270718DE0618092004C603183ABDF1CFDE2709099C5D2405861C7EEAEF99
S123F4A0DF271AEF0018387EF43BDE279C5F2605861D7EEAEF1AEE000808DF2739CEF4DC22
S123F4C0BDE11CDC29BDEB1A18DF312007BDE1108601971CCC0000DD297EE0160A0D53546C
S123F4E04F50504544204154204C494E4520232000DE2509099C592405861E7EEAEFDF25FE
S123F5001AEF00C6013718DE2B260139183C189C0627BADE2BE6023ADF2BC603183ABDF172
S123F520CF18A600183833811926015C811A26D55A26D27EF47ADE259C5B2605861F7EEA94
S123F540EF183C1AEE00BDFB17BDFBBE260A1838DE250808DF252002313139BDFB17BDF146
S123F560CF18A600361808BDF1CFDE1FEC002A07260586207EEAEFEC008300012717ED004A
S123F580C603183ABDF1CF18A600817D27E41808BDF1CF20E2BDFBBE32811226037EF43B58
S123F5A0183CC603183ABDF1CF18A600817D270B817A27071808BDF1CF20E77EF49018087E
S123F5C0BDF1CFBDFB17BDF1CF1808BDF1CFBDFB171808BDFBBE8FBDFBBE8FE70039C600E2
S123F5E0DE613A3C1808BDFB17BDFBBE4D2705862E7EEAEF38E70039C60420E4C60320E07A
S123F600C60820DC86FF971B397F001B390F07847F06CF078A80060E39BDF85718A6008142
S123F6207D2704817A2607BDE1107F00373981A22616183CC60218EB01183A3808E600C0A2
S123F640020808BDF8D520398136261E18A60181072605BDF6BE202981022605BDF6D32036
S123F66020810B2605BDF6E7201781122605BDF6DF200EBDFB17BDFBBEBDEB1A8620BDFEF8
S123F680D2BDF1CF18A600817C2708817B2628180820131808D61EC40750CB0827088620B9
S123F6A0BDFED25A26FABDF1CF18A600817D270A817A27067EF62EBDE1107F0037398D439E
S123F6C02705862A7EEAEFD11E23078620BDFED220F5398D2E2704862B20E9177EFED28DC7
S123F6E0222708863220DD8D1A8D0117368D0332200444444444840F8B30813923028B07C9
S123F7007EFED2C603183ABDFB171808BDFBBE4D3918A6008510260586217EEAEF18EC0110
S123F720D3088FEC032704862220EF3CC604183ABDFB17180838DC2DED03C30002DD2DBD86
S123F740FBBE2A04862720183CEE03ED00C300013805D32D1A932D23051A93102305860948
S123F7607EEAEFDD2DEE0308086F00089C2D26F9BDF1CF18A600817D27071808BDF1CF20A0
S123F7809039DC2383000A1A9355240586237EEAEFDD23183CBDF4041838DE23ED00DC2999
S123F7A0ED08BDF3F1BDF1CF1808BDF1CFBDFB17BDFBBEDE23ED04CC0001ED02BDF1CF180D
S123F7C0A600813A27041AEF06391808BDF1CFBDFB17BDFBBEDE2320E1BDF404DE231AA3FA
S123F7E000270586247EEAEF183C1AEE0018EC00E30218ED006D022B111AA3042F11183892
S123F8008FC3000ADD23BDF1CF391AA3042DEF18381AEE06EC08DD29398D3C18A60081A2BA
S123F820261B183CC60218EB01183A3808E600C0020808BDF8D51808BDF1CF2003BDE11021
S123F840CEF854BDE11CBDE0BB8D3B25F0BDE1107F0037393F200018A6008178270139186F
S123F86008BDF1CFBDFB17BDFBBE2A0586307EEAEF1A83000722F5D737BDF1CF817D27050E
S123F8801808BDF1CF39BDE05B810D26020D398D17BDF1CF18A600817D270B817A2707184A
S123F8A008BDF1CF20E00C3981242608BDE3CCBDE6CF2003BDF8E23736BDE05B812C2709CD
S123F8C0810D270886157EEAEFBDE3CCBDF4048F3233ED00395D2709A60008BDFED25A26F2
S123F8E0F739BDE3C3812D260CBDE3CCBDE6A14353C3000139BDE6A139DE3326048D1DDE0E
S123F90033DF00BDF8862505DE00DF3339183C18DE00180818088D3A183820DD183C18DE5B
S123F92004183C18E602183A18DF331838C603183ABDF1CF18A600810C270D18DE33189CAB
S123F9400626DE86267EEAEF1808180818DF33183839183C20E8BDFB17BDF1CF1808BDF12D
S123F960CFBDFBBE27037EF43BC603183ABDF1CF18A600813926071808BDF1CF20E8391834
S123F98008BDF1CFBDFB1718081808BDFB17183C18DE1F18EC022B061A8300FF23058628EE
S123F9A07EEAEF05C3B6008FA60081FF27028D1D08A60081FF27028D1418A6018D3209184F
S123F9C0A6008D2C1838BDFBBEBDFBBE39183C18DE61C61618E73BA70007360FC61718E7BF
S123F9E03B8D36C61618E73B3206186F3B183839183C18DE61C60218E73BA7003607360F96
S123FA00C60318E73B8D12C60218E73B3206186F3B32A10026DF1838393CCE0D020926FD9E
S123FA203839BDF857BDF4048FBDFEEF164FED007F0037391808BDFB17BDFBBEDD38390F54
S123FA408603973CDE61EC0EBDEE054F5FDD380E391808BDFB17BDFBBE4D270586357EEA52
S123FA60EFDE61E727398D4ABDFB17BDFBBEDD3ABDF1CF1808BDF1CF18DF3D20198D33BDD6
S123FA80FB17BDF1CF1808BDF1CFBDFBBE2604DD3F200318DF3FC603183A398D150785108F
S123FAA0260586347EEAEFDC45DD29DC47DD2B31313B7D0019270586337EEAEF398DF3BDCF
S123FAC0FB17BDF1CF1808BDF1CFBDFB17BDF1CF1808BDF1CF07360F18DF41BDFBBE1A8376
S123FAE00001230586367EEAEF86105D270148DE61A724BDFBBE2608DE616F26DD41201093
S123FB001A83000422DECB0358585858DE61E7263206C603183A398610BDFC2018A600818C
S123FB2010260818088DF0180820F14D2A048D1220EABDFBCDBDFC102401391808BDFC20EC
S123FB4020DA8184260E18EC01D3088FC603183AEC03202D81A4260DCDEE01C60418EB03C4
S123FB60183A8F201C819426138D2A183C3C05183018E3003818388FEC00200586087EEA69
S123FB80EFDE1F09099C512407861797187EEAEFDF1FED003918EC01D3088FEE0326058673
S123FBA0187EEAEFC604183A3CBDFB17180838BDFBBE1AA3002304861920E60808393CDEF1
S123FBC01FEC000808DF1F381A83000039813627013918A6014AC603183A1658CEFBEA3A63
S123FBE0EE00AD00180818A60039FE25FEA3FE4AFDCDFE7BFDDEFEA3FDF0FDFBFE0AFEA3F6
S123FC00FEB3FEC2FEC6FECAFECEFEA8FEA3FEAC81112708817A24020C3986118D020D3993
S123FC20DE21099C4D260586177EEAEFDF21A700DE21A60081102719E601C4F084F0112251
S123FC4010A601E600C1112609811026050808DF2139E70108DF218D0220D58170250780EC
S123FC6070CEFCA9203C816025078060CEFCAF2031815025078050CEFCB12026814025070F
S123FC808040CEFCB7201B813025078030CEFCBB2010812025078020CEFCC7200586087E73
S123FCA0EAEF16583AEE006E00FD85FD86FD8FFDCCFD57FD05FD51FCEFFCF8FD97FDA2FD56
S123FCC0A8FDAEFDB4FDBAFCE4FCD9FCCDBDFBBEDE1FA800E801ED0039BDFBBEDE1FAA00A0
S123FCE0EA0120F2BDFBBEDE1FA400E40120E7BDFBBEDE1FE30020DEDE1FEC02A30008080E
S123FD00ED00DF1F398D08BDFBBEDE1FED0039DE1FA600A80236EC002605861A7EEAEF2AD2
S123FD2003BDFD8F6D022A09EC024353C30001ED02EC00EE028F023CDE1FED023233ED00B3
S123FD40324D2A0CBDFD8FEC024353C30001ED02398DBCBDFBBE39183CDE1FA601E6033D1B
S123FD6037361830A601E6023D18EB0018E700A600E6033D18EB0018E70008083233ED00CC
S123FD80DF1F18383939DE1FEC004353ED00398DF5C30001ED00398D272C026C030808DF4E
S123FDA01F398D1C2FF720F38D162EF120ED8D102DEB20E78D0A26E520E18D0427DF20DB45
S123FDC0DE1FEC026F026F031AA3003939BDFB17DE1FEC002A054353C30001ED0039BDFB03
S123FDE017DE1FEC0027F4CC00016D002AED20E6BDFB17DE1FEE00AD00200ABDFB17DE1F30
S123FE00EE00E6004FDE1FED0039BDFB17DE1FEC001A8300FF230586287EEAEF05C3B60099
S123FE208FEC0020E0BDFB17BDF1CF1808BDF1CFBDFB17DE1FEC02EE00032804862C20D9D8
S123FE408FDE1F0808ED00DF1F39BDFB17DE1FEC002B061A8300072304862D20E1DE61E750
S123FE60306D302AFC4FE631EB328900EB338900EB3489000404DE1FED0039BDFB17DE1F39
S123FE80EC00270C2B04DC352015DE61EC0EDD35DC35581BD6360505D335C33619DD3504B5
S123FEA0ED003986297EEAEFDC38200FDE61E6274F2008C600DE613AE6004F180918097ED8
S123FEC0FB81C60420EFC60320EBC60820E7C60A20E37C001E373CCE00B4D637583AEE0031
S119FEE026087F003786317EEAEFAD00383339373CCE00A420E4DC
S123FF008D0D36B69800850227F932B7980139B69800850127F9B698013936B698008501D7
S123FF2032393CDE61A62E842027FAA62F38393CDE6136A62E858027FA32A72F38393CDEBA
S123FF406136A62E85203238398D2A8D11867E979E97A1CCFF1ADD9FCCFF0FDDA2393CDE17
S123FF60618630A72B6F2C860CA72D861197438613974438398613B798008656B7980039F1
S117FF808DBC270E368D9B914426068D95914326FA32209B89
S123FFA0FF00FF22000000000000000000000000FF02FF800000000000000000000000009D
S113FFC0C0002000600020001000F424FF4940001D
S123FFD600C400C700CA00CD00D000D300D600D900DC00DF00E200E500E800EB00EE00F15F
S10DFFF600F400F700FA00FDED77B7
S903E00319
